:03000000023F7745
:0C3F770078FFE4F6D8FD758175023FBEAE
:1014980020000A3C2E2E2E3E004950436F6E6E658A
:1014A80063745245510A004950436F6E6E65637408
:1014B800000A49504E6F41434B210A003E432C56C7
:1014C8002C52432CC0E4E0EFF2E5F020D1E8EDEA3D
:1014D800EEEC49500A003E432C4D41432C25303256
:1014E80062583A25303262583A25303262583A25E5
:1014F800303262583A25303262583A2530326258D2
:101508002C4D414320E0E4F0E5F10A003E432C561F
:1015180045522C20332E3220EEF2202573202573DD
:101528002CC2E5F0F1E8FF20495020ECEEE4F3EBA3
:10153800FF0A004A756E20333020323030380031CF
:10154800323A30393A3036003E432C4C442C505213
:101558004F473A2020202020202020202020202013
:101568002020202020202020202020202020202073
:101578002020202020202020202020202020202063
:101588002020202020202020202020202020202053
:1015980020202020202020202CC4E0F2E020EFF0A2
:1015A800EEF8E8E2EAE828F4E0E9EB290A003E2A46
:1015B8002C312CCEF1EDEEE2EDFBE520EFE0F0E092
:1015C800ECE5F2F0FB20F1E5F2E5E2EEE3EE20E8EF
:1015D800EDF2E5F0F4E5E9F1E00A003E412C413096
:1015E800312C2562752E2562752E2562752E256291
:1015F800752C495020E0E4F0E5F120E0E4E0EFF25A
:10160800E5F0E00A003E412C4130322C2562752E6F
:101618002562752E2562752E2562752C495020E0AD
:10162800E4F0E5F120EEF1ED2E20F1E5F0E2E5F051
:10163800E00A003E412C4130332C2562752E25628C
:10164800752E2562752E2562752C495020E0E4F030
:10165800E5F120F0E5E72E20F1E5F0E2E5F0E00A1B
:10166800003E412C4130342C2562752E2562752EA2
:101678002562752E2562752CCCE0F1EAE020F1E5B3
:10168800F2E80A003E412C4130352C2562752E25A2
:1016980062752E2562752E2562752CD8EBFEE70A39
:1016A800003E2A2C312CC4EEEF2E20EFE0F0E0ECC7
:1016B800E5F2F0FB20F1E5F2E5E2EEE3EE20E8EDFD
:1016C800F2E5F0F4E5E9F1E00A003E422C5330314E
:1016D8002C2562752CC6E4E0F2FC20E7E0EFF0EE82
:1016E800F1E020F1EEE5E4E8EDE5EDE8FF20EEF2CB
:1016F80020F1E5F0E2E5F0E00A003E422C533032FA
:101708002C2562752CCEE1ECE5ED20F120F1E5F019
:10171800E2E5F0EEEC20E1E5E720EAE2E8F2E0EDD0
:10172800F6E8E90A003E422C5330332C2562752C2A
:10173800CFE5F0E5E7E0EFF3F1EA20EFF0E820EF9E
:10174800EEF2E5F0E520F1E2FFE7E820F120F1E52F
:10175800F0E2E5F0EEEC0A003E422C5330352C2541
:1017680062752CCAE0EDE0EB20F8E8F0EEEAEEE274
:10177800E5F8E0F2E5EBFCEDEEE3EE20EEE1ECE57A
:10178800EDE00A003E532C5330362C253032625897
:101798002530326258253032625825303262582559
:1017A8003032625825303262582C4D414320E0E4F3
:1017B800F0E5F120F8E8F0EEEAEEE2E5F8E0F2E52F
:1017C800EBFCEDEEE3EE20EEE1ECE5EDE00A003EA9
:1017D800454E440A000A44756D7058202020202088
:1017E8003030203031203032203033203034203037
:1017F80035203036203037203038203039203041FD
:101808002030422030432030442030452030460AE2
:10181800000A3A003A20000A000A44756D70442014
:10182800202020203030203031203032203033202A
:1018380030342030352030362030372030382030D2
:101848003920304120304220304320304420304578
:1018580020304600457272206B657900526420651D
:101868006570726F6D0A005264204D454D0A005232
:101878006420436F64650A00577269746520436F7A
:1018880064650A0044656275674950204F4E0A0036
:1018980044656275674950204F46460A00446562B0
:1018A800756755736572204F6E0A004465627567E7
:1018B80055736572204F46460A0044656275674D48
:1018C8007367204F6E0A0044656275674D73672021
:1018D8004F46460A00436F6E666967206C6F636BFC
:1018E800210A00577220656570726F6D0A002053D7
:1018F80061766520656570726F6D210A00457272A8
:10190800204D414321004C6F61643E3E002A003C5B
:101918004130313D003C4130323D003C4130333DA7
:10192800003C4130343D003C4130353D003C210015
:101938003C5330313D003C5330323D003C53303352
:0E1948003D003C5330353D003C5330363D00F1
:063C3D000113000111005B
:10496A00C28E438910E4F58B758DB8D2ABD28E22F4
:03001B00023EE7BB
:103EE700C0E0C083C082C0D0C28E758B00758DB80C
:103EF700201C0675A61E75A6E10511D218E51360EC
:103F0700020513E512D39401400215120516E516B2
:103F1700540F7048D224E516543F7012D21690669B
:103F27008BE0600A04F0E0D394B44002D21C9066A0
:103F370086E0600204F0906104E0600214F090668D
:103F47008CE0D394014003E014F0301B020514E524
:103F570015D394644004D21C80020515E510D39450
:103F67000140021510D28ED0D0D082D083D0E0325B
:10090E00C2AFC2217D027C007F071249338F45E5BD
:10091E0045646060097D017F601248CBD221E4FD01
:10092E00FC7F0B1249338F45E54530E6097D04E423
:10093E00FF1248EFD2217D017C007F071249338FD1
:10094E0045E5457008FD7FFF1248CBD221302103CB
:10095E00126000C288C2A8C2AA758900123E4B90CE
:10096E0063497403F0A374CCF0E4906348F0123B37
:10097E0073122BE6C21C12459CD221C223C22290B6
:10098E0065767408F09062B47424F0E4A3F090637A
:10099E003EE09062B6F090633FE09062B7F09063F5
:1009AE0040E09062B8F0906341E09062B9F09063DD
:1009BE0042E09062BAF0906343E09062BBF0751231
:1009CE0001E4906577F0C21DC21EC21FC220202115
:1009DE0018AF45FE7D031238DEE4FF123CFD7E1497
:1009EE007F98E4FBFDFC1234F990668BE060037493
:1009FE0001F0E4906104F0F514906575F0F51512B0
:100A0E00496A75A70775A61E75A6E1D2AFE4F5155E
:100A1E00906104E07003120ED790668CE0B4011161
:100A2E009080007410F0E490668CF0D221C222C245
:100A3E0023908008E0F54530E405D21D7410F0E5F2
:100A4E004530E508D21F9080087420F0E54530E669
:100A5E0008D21E9080087440F0E514C39403401928
:100A6E00908002E4F0908001F0908000F0E5149404
:100A7E00064006E4F51412459C9080A0E070031227
:100A8E0043209080B8E0700312439A9080D0E070BB
:100A9E000312447E908000E07013301D1012360059
:100AAE00906331EFF0D39400400312003690800231
:100ABE00E07006908000E06005D21B020A1BC21B8C
:100ACE00E4F514906104E06003020A1B20211290E9
:100ADE006578E0600C7E147F9A1237F6E4906578A4
:100AEE00F0301F1212324E906331EFF0D39400406B
:100AFE0005E0FF120032201E03020C7F122F4A90D7
:100B0E006331EFF07003020A1B906375E054BF244B
:100B1E007F7003020BE8147003020BC02402600303
:100B2E00020C212021077E147FA11237F620250307
:100B3E00020C7F90634DE0FF7006906351E06061A0
:100B4E00906682E0FEB50722A3E0FF90634EE0B50B
:100B5E000718906684E0FF90634FE0B5070C90662F
:100B6E0085E0FF906350E06F6037906351E06E60F8
:100B7E0003020C7F906683E0FF906352E06F600388
:100B8E00020C7F906684E0FF906353E06F60030277
:100B9E000C7F906685E0FF906354E06F6003020C5B
:100BAE007FC2199065777401F01249CD751201025A
:100BBE000C7F90668BE060037401F090667AE0FF24
:100BCE00906377E06F6003020C7F90667AE004F02A
:100BDE00E4F512906575F0020C7F301903020C7F5C
:100BEE00906344E07003020A1B906355740AF0127E
:100BFE0047F2D219E4F512906575F090668604F00E
:100C0E00E4906679F0A3F02021677E147FAF12374F
:100C1E00F6805E90668BE060037401F0301952909E
:100C2E006375E020E74B906377E0FF906679E0FE16
:100C3E006F600D906681E07007EE146F7033801355
:100C4E00906679E004F0906331E0FFD394044003A2
:100C5E00123DAD9060007482F0A37401F090637742
:100C6E00E0906002F07E607F007D0312408A020AEF
:100C7E001B201903020D97E5127068124789EF6069
:100C8E00237E647F75906476E02404FD12408A9082
:100C9E006681E07009906355E0F512020A1BE4F5D7
:100CAE0012020A1B906686E0D3943C403690668111
:100CBE00E0703090668604F0123A9AE4906475F013
:100CCE00A37412F090667AE0906477F0A374FDF04E
:100CDE0090610563A20190647963A2017F12122ACA
:100CEE00D8809E1249BB8F45E545B4011590600032
:100CFE007483F0E4A3F07E607F007D0212408A02CE
:100D0E000A1BE545D39401401C9060007483F0A348
:100D1E007401F0E54524FEA3F07E607F007D031292
:100D2E00408A020A1BE51264016003020A1B9065E9
:100D3E0075E004F02021077E147FB91237F6906318
:100D4E0055E0C394C85004E02432F0906575E0C3BA
:100D5E009405400DC219E4906577F01249CD020A50
:100D6E001B7C667D82906349E0FAA3E0FB7F021252
:100D7E00421B7E647F75906476E02404FD12408AE7
:100D8E00906355E0F512020A1BE51264016003023E
:100D9E000A1B906577E014604624FE6042147003CF
:100DAE00020E8A24046003020A1BE4F514202513A4
:100DBE009065777404F0906575E05401F07512013A
:100DCE00020A1B9080027410F0E4906577F0906533
:100DDE007504F07512FA90668274FFF0020A1B9089
:100DEE006682E07003020E749064757480F09064F5
:100DFE00777401F0E4A3F0A304F0A37430F0A374AD
:100E0E007BF0E4F545747C2545F582E43464F58386
:100E1E00747DF0747D2545F582E43464F583E4F049
:100E2E00E5452407906476F07C667D82906349E008
:100E3E00FAA3E0FB7F0212421B7E647F75E5452418
:100E4E0009FD12408A906681E0601B1247F2D219AA
:100E5E00E4F512906575F090668604F0E49066797C
:100E6E00F0A3F0020A1B302507E4906577F08006A8
:100E7E009065777404F07512FA020A1B9080027462
:100E8E0010F0751205906575E06401FFF0906577BE
:100E9E007401F0EF7019906351E06013FCA3E0FD54
:100EAE00A3E0FEA3E0FF9066821226B2020A1B9018
:100EBE00634DE0FCA3E0FDA3E0FEA3E0FF9066829D
:080ECE001226B2020A1B80FE8D
:010ED60022F9
:10003600906376E0B444047F0180027F009063758C
:10004600E0B447047E0180027E00EE5F604A906362
:100056003EE0906377F090633FE0906378F09063C2
:1000660040E0906379F0906341E090637AF09063AA
:1000760042E090637BF0906343E090637CF0906392
:10008600767452F09062AE63A2019080A863A201DA
:100096007F06122AD8020904906331E0C3940850FF
:1000A6000302090D90633EE0FF906377E06F600303
:1000B60002090D90633FE0FF906378E06F600302F2
:1000C600090D906340E0FF906379E06F60030209D9
:1000D6000D906341E0FF90637AE06F600302090DC3
:1000E600906342E0FF90637BE06F600302090D902E
:1000F6006343E0FF90637CE06F600302090D906349
:1001060076E0B444159062AEE0B4FF0E63A20190AF
:1001160080A863A2017F06122AD890668BE060034E
:100126007401F090668C7464F09063767452F0906B
:100136006375E0646D60030202957BFF7A1479C4EF
:1001460012221E7BFF7A1479DE90633EE0F54EA301
:10015600E0F54FA3E0F550A3E0F551A3E0F552A377
:10016600E0F55312221E754EFF754F1575503B75FF
:1001760051FF7552157553477BFF7A157914122274
:100186001E7BFF7A15795012221E7BFF7A1579B6EF
:1001960012221E7BFF7A1579E3906344E0F54EA3A5
:1001A600E0F54FA3E0F550A3E0F55112221E7BFFC8
:1001B6007A16790D90634DE0F54EA3E0F54FA3E076
:1001C600F550A3E0F55112221E7BFF7A16793B907B
:1001D6006351E0F54EA3E0F54FA3E0F550A3E0F53B
:1001E6005112221E7BFF7A16796990633AE0F54E2A
:1001F600A3E0F54FA3E0F550A3E0F55112221E7BD4
:10020600FF7A16798C906336E0F54EA3E0F54FA39E
:10021600E0F550A3E0F55112221E7BFF7A1679A96C
:1002260012221E7BFF7A1679D2A225E433F54E12EE
:10023600221E7BFF7A177902906681E0F54E122224
:100246001E7BFF7A17792D90668BE0F54E12221EE3
:100256007BFF7A177960A217E433F54E12221E7BD4
:10026600FF7A17798C90667BE0F54EA3E0F54FA3F5
:10027600E0F550A3E0F551A3E0F552A3E0F55312E3
:10028600221E1233B47BFF7A1779D712221E2290D0
:100296006375E0644C60030203547E177FDDFBFD4B
:1002A600FC1234F990637DE0F546A3E0F547E4F5EA
:1002B60049E4F548854782854683E0FF747F2548F3
:1002C600F582E43463F583EFF00548E548B410E4BD
:1002D600E54690637FF0A3E547F07E187F197C63BF
:1002E6007D7F7B021234F9E4F54885478285468393
:1002F600E0FF747F2548F582E43463F583EFF0056B
:1003060047E547700205460548E548B410DC7E1807
:100316007F1C7C637D7F7B101234F9E4F5488547AA
:1003260082854683E0FF747F2548F582E43463F5D1
:1003360083EFF00548E548B410E40549E549C39460
:100346001050030202B77E187F1F1237F622906301
:1003560075E0646C60030203F5F54A7E187F21FBA5
:10036600FDFC1234F9E4F549E4F548A84AE6FF74C1
:100376007F2548F582E43463F583EFF00548E548C8
:10038600B410E8E490637FF0A3E54AF07E187F1985
:100396007C637D7F7B021234F9E4F548A84AE6FFC8
:1003A600747F2548F582E43463F583EFF0054A054A
:1003B60048E548B410E67E187F1C7C637D7F7B1081
:1003C6001234F9E4F548A84AE6FF747F2548F58219
:1003D600E43463F583EFF00548E548B410E80549D1
:1003E600E549C3940840817E187F1F1237F6229094
:1003F6006375E0644B7061F54874672548F582E4DF
:100406003463F583E0603274672548F582E434632B
:10041600F583E0F4602374672548F582E43463F5D8
:1004260083E0FF747D2548F582E43463F583E0B507
:1004360007100548E548B408C09061047432F0021C
:1004460009049063757421F03021030209047E18B3
:100456007F5C1237F6020904906375E0B4521A20E5
:1004660021077E187F641237F69063757472F07EEA
:10047600637F757D0812400322906375E0644970BE
:10048600452021077E187F6F1237F690637DE0F5D1
:1004960046A3E0F547E4F548854782854683E0FFB5
:1004A600747F2548F582E43463F583EFF00547E56C
:1004B60047700205460548E548B480DC7E637F75D3
:1004C6007D8A12400322906375E0644370462021C2
:1004D600077E187F771237F690637DE0F546A3E036
:1004E600F547E4F548854782854683E493FF747FA4
:1004F6002548F582E43463F583EFF00547E5477058
:100506000205460548E548B480DB7E637F757D8A33
:1005160012400322906375E0645A70532021077ECF
:10052600187F801237F690637DE0F546A3E0F54725
:100536007C637D7F7B80AF47AE461247BEE4F548BD
:10054600854782854683E493FF747F2548F582E4D8
:100556003463F583EFF00547E54770020546054825
:10056600E548B480DB7E637F757D8A124003229066
:100576006375E06444600302060690637DE0FF64F1
:10058600447003020904EFB4310CC2217E187F8C3B
:100596001237F602090490637DE0B4300CD2217E56
:1005A600187F981237F602090490637DE0B4320C86
:1005B600D2227E187FA51237F602090490637DE0E9
:1005C600B4330CC2227E187FB31237F602090490A8
:1005D600637DE0B4340CD2237E187FC21237F60254
:1005E600090490637DE0B4350CC2237E187FCF12D8
:1005F60037F602090490637DE0FF12001E0209042B
:10060600906104E070132021077E187FDD1237F613
:100616009063757421F00209049061047432F090BD
:100626006375E0FFB45104C2AF80FEEF64577045B6
:100636002021077E187FEB1237F690637EE09063E9
:1006460031F0E4F548906331E0FFE548C39F40038D
:10065600020904747F2548F582E43463F583E0FFDC
:1006660090637DE0254824ADF582E43461F583EF9F
:10067600F0054880D0906375E06453600302072854
:100686002021077E187FF61237F690633EE0FF9032
:1006960061B6E06F703C90633FE0FF9061B7E06F3A
:1006A6007030906340E0FF9061B8E0B50724906336
:1006B60041E0FF9061B9E0B50718906342E0FF9012
:1006C60061BAE0B5070C906343E0FF9061BBE06F51
:1006D60060169063757421F03021030209047E19B7
:1006E6007F051237F6020904E4F548E4F51574AD02
:1006F6002548F582E43461F583E0FDAF48124851A0
:100706000548E548C394FE40E2C2AFE4907FF0F0AE
:10071600A3F0907FFD74AAF0A374FFF0A37455F0C4
:1007260080FE906375E0644F704C90637DE0F54603
:10073600A3E0F547E5474546700A2021077E197F65
:100746000E1237F62021077E197F151237F6E4F5CB
:1007560048747F2548F582E43463F583E085478253
:10076600854683F00547E547700205460548E54896
:10077600B480DE020904906375E0FFB445219063FE
:100786007DE0FDA3E0907FF0CDF0A3EDF0C2AF9049
:100796007FFD74AAF0A374FFF0A37455F080FEEFFA
:1007A6006465600302090D90637DE0FFA3E0907F1E
:1007B600F0CFF0A3EFF0E4F546F547D3907FF1E0F4
:1007C6009547907FF0E095464021E4F5152547FFD3
:1007D600E5463478FE7B80AD47AC461247BE748052
:1007E6002547F547E43546F54680D07E197F171232
:1007F6004111EF4E6020120003906344EFF01200A7
:1008060003906345EFF0120003906346EFF0120089
:1008160003906347EFF07E197F1D124111EF4E6082
:100826002012000390634DEFF012000390634EEF29
:10083600F012000390634FEFF0120003906350EF45
:10084600F07E197F23124111EF4E602012000390B3
:100856006351EFF0120003906352EFF01200039021
:100866006353EFF0120003906354EFF07E197F2973
:10087600124111EF4E602012000390633AEFF0121E
:10088600000390633BEFF012000390633CEFF0121D
:10089600000390633DEFF07E197F2F124111EF4E5A
:1008A6006020120003906336EFF012000390633766
:1008B600EFF0120003906338EFF0120003906339F3
:1008C600EFF0E4F548E4F515E54804FF74362548ED
:1008D600F582E43463F583E0FD1248510548E548A6
:1008E600C3944340E0C2AFE4907FF0F0A3F0907F62
:1008F600FD74AAF0A374FFF0A37455F080FE7E6326
:070906007F757D081240031C
:01090D0022C7
:10475100AE07EEC39430400BEED394395005EE24EE
:10476100D0FF22EEC39461400BEED394665005EE68
:1047710024A9FF22EEC39441400BEED39446500589
:08478100EE24C9FF22AF06225D
:104950009062ADE004F070069062ACE004F090620A
:0A496000ACE0FEA3E0FF1246952232
:10000300124950124751EFC454F0FEC00612495032
:08001300124751D0E02FFF223B
:10453F00E4906B1FF0124950906B20EFF0C3943052
:10454F004018E0FFD394395011906B1FE02405F50C
:10455F0082E43461F583EFF08011906B1FE0240546
:10456F00F582E43461F583E4F0800C906B1FE00476
:10457F00F0E0D3940840BE75540075550075560091
:0C458F00E4F5577B017A617905122DA636
:01459B0022FD
:044111008E4B8F4CF6
:104115009062ACE4F0A374FFF0124950EF606EF4C6
:10412500606B854C82854B83E493B507EC754D0137
:10413500E54C254DF582E4354BF583E493602590F8
:1041450062ADE0254DFF9062ACE03400FE1246956D
:10415500E54C254DF582E4354BF583E493B507042D
:10416500054D80CCE54C254DF582E4354BF583E4D2
:104175009370A6E54D24FFFFE434FFFE9062ADE0A9
:104185002FF09062ACE03EF07E007F0122E4FEFF5E
:014195002207
:103B73007E197F35124111EF4E70037F01227E19AA
:103B83007F38124111EF4E600C124950EF24D024BC
:103B9300FF92258002D2257E197F3E124111EF4EFE
:103BA300600C124950EF24D0906681F08005E490B8
:103BB3006681F07E197F44124111EF4E600C124969
:103BC30050EF24D090668BF08005E490668BF07EF6
:103BD300197F4A124111EF4E600C124950EF24D065
:103BE30024FF92178002C21790633E63A20190667E
:103BF3007B63A2017F06122AD830173B7E197F50C0
:103C0300124111EF4E603012000390667BEFF01209
:103C1300000390667CEFF012000390667DEFF012D4
:103C2300000390667EEFF012000390667FEFF012C0
:0A3C33000003906680EFF07F00228E
:10464E00906576E0C3947C503D906576E0FE04F074
:10465E0074B42EF582E43462F583EFF0BF0A27902E
:10466E006576E0FF04F074B42FF582E43462F583CE
:10467E00E4F0906576E0FF1241969065767408F04E
:07468E009062B5E004F02288
:10459C009080007480F090633663A201F583F582FD
:1045AC0063A2017F08122AD890633E63A201908017
:1045BC008863A2017F0A122AD8908092E4F0A37437
:1045CC0032F0A37401F0906348E0FF9080B1F0905A
:1045DC0080E1EFF09080957455F0A3F0908000741A
:0945EC0001F090800974F0F02246
:10432000908009E04410F09080A0E0706C9080A133
:104330007482F09080A874FFF0A3F0A3F0A3F07F44
:10434000039080AEEFF07FCBA3EFF07F039080ACC3
:10435000EFF0A374CBF09080007402F0906B0E121B
:1043600026BE00000000906B0EE0908040F0906B45
:104370000FE0908041F0906B10E0908042F0906BE5
:1043800011E0908043F0A3E4F0A3F0A3F0A3F09039
:094390008018F0A3F0A3F0A3F0E3
:014399002201
:10447E00908009E04440F09080D17482F0906349BE
:10448E00E0FF9080DEF090634AE0FF9080DFF090D6
:10449E0080027402F0906B121226BE000000009093
:1044AE006B12E0908058F0906B13E0908059F09072
:1044BE006B14E090805AF0906B15E090805BF0A347
:1044CE00E4F0A3F0A3F0A3F0908030F0A3F0A3F0FB
:0244DE00A3F049
:0144E00022B9
:10439A00908009E04420F09080B8E0706C9080B979
:1043AA007482F07F039080C6EFF07FCDA3EFF07F99
:1043BA00039080C4EFF0A374CDF09080C074FFF036
:1043CA00A3F0A3F0A3F09080017402F0906B161290
:1043DA0026BE00000000906B16E090804CF0906BB7
:1043EA0017E090804DF0906B18E090804EF0906B43
:1043FA0019E090804FF0A3E4F0A3F0A3F0A3F090AB
:09440A008024F0A3F0A3F0A3F05C
:014413002286
:10421B008C468D47A907EAFDE975F018A424ACFF7D
:10422B00E5F034808F82F583EDF0EBFDE975F01846
:10423B00A4FFAEF024ACFBEE34808B82F583A3EDB0
:10424B00F08547828C83E0FDEF24A8FFEE3480FEDF
:10425B008F82F583EDF08547828C83A3E08F828E6E
:10426B0083A3F0854782854683A3A3E0FDE975F020
:10427B0018A424A8FFE5F03480FE8F82F583A3A356
:10428B00EDF08547828C83A3A3A3E08F828E83A35B
:04429B00A3A3F022C7
:064003008D4BAB07AA067D
:10400900908000E030E5079065787401F022906BAC
:104019000EE0FCA3E0FDA3E0FEA3E0F54F8E4E8D7C
:104029004D8C4CAE02AF038E838F8263A201E54EA5
:10403900540744C0F583854F8263A201AF4B122B0D
:104049004AE4FCFDFEE54F254BF54FEE354EF54EA6
:10405900ED354DF54DEC354CF54C908040E54CF087
:10406900A3E54DF0A3E54EF0A3E54FF09080007471
:1040790020F0AF4FAE4EAD4DAC4C906B0E1226B248
:014089002214
:06408A008D46AB07AA06FB
:10409000908002E030E5079065787403F022906B21
:1040A00012E0FCA3E0FDA3E0FEA3E0F54A8E498DFB
:1040B000488C47AE02AF038E838F8263A201E5492D
:1040C000540744D0F583854A8263A201AF46122B80
:1040D0004AE4FCFDFEE54A2546F54AEE3549F54938
:1040E000ED3548F548EC3547F547908058E547F001
:1040F000A3E548F0A3E549F0A3E54AF090800274F7
:1041000020F0AF4AAE49AD48AC47906B121226B2D0
:01411000228C
:023CFD008F46F0
:103CFF00908001E030E5099065787402F07F002232
:103D0F00906B16E0FCA3E0FDA3E0FEA3E0F54A8E66
:103D1F00498D488C4790667B63A201E5495407445F
:103D2F00C8F583854A8263A2017F06122B60E54A9C
:103D3F002406F54AE43549F549E43548F548E435B4
:103D4F0047F54790657963A201E549540744C8F5E3
:103D5F0083854A8263A201AF46122B60E4FCFDFE0D
:103D6F00E54A2546F54AEE3549F549ED3548F5481A
:103D7F00EC3547F54790804CE547F0A3E548F0A3B5
:103D8F00E549F0A3E54AF09080017420F0AF4AAE08
:0D3D9F0049AD48AC47906B161226B2AF46F6
:013DAC0022F4
:103600009081E0E0F5460546054605460546054637
:1036100005460546054605460546908010E0F549F5
:10362000A3E0F54AA3E0F54BA3E0F54C9081E1E07F
:10363000F546054605460546054605460546054642
:10364000054605460546908014E0F54DA3E0F54E8D
:10365000A3E0F54FA3E0F550E54FB54B08E550B5B5
:103660004C037F0022E4F546E54F540744E0F58320
:1036700085508263A20190637563A2017F08122BBB
:103680009090637763A2019062AE63A2017F0612FD
:103690002AD8906375E0F547A3E0F548E4F5469035
:1036A0006375E0702AA3E024F8F546E54F5407441B
:1036B000E0F58385508274082582F582E43583F530
:1036C0008363A20190637563A201AF46122B90AE93
:1036D00047E4FCFDE5502548F550E54F3EF54FED3C
:1036E000354EF54EEC354DF54D908014E54DF0A37B
:1036F000E54EF0A3E54FF0A3E550F0908000744054
:03370000F0AF46E1
:0137030022A3
:102F4A009081E6E0F54605460546054605460546EE
:102F5A0005460546054605460546908028E0F5499A
:102F6A00A3E0F54AA3E0F54BA3E0F54C9081E7E036
:102F7A00F5460546054605460546054605460546FF
:102F8A0005460546054690802CE0F54DA3E0F54E32
:102F9A00A3E0F54FA3E0F550E4F546E54FB54B0A3B
:102FAA00E550B54C05C21E0230B6E54F540744F051
:102FBA00F58385508263A20190637563A2017F083D
:102FCA00122B90906375E0F547A3E0F548E5484574
:102FDA004770099080027410F07F0022906682E0A8
:102FEA00FFF46030906377E06F600302307D906693
:102FFA0083E0FF906378E06F7079906684E0FF90D9
:10300A006379E06F706D906685E0FF90637AE06F98
:10301A006031805F906377E0906682F0906378E039
:10302A00906683F0906379E0906684F090637AE02A
:10303A00906685F090637BE0FFA3E0906349CFF050
:10304A00A3EFF0906375E0702AA3E024F8F546E553
:10305A004F540744F0F58385508274082582F5821F
:10306A00E43583F58363A20190637563A201AF46D9
:10307A00122B90AE47E4FCFDE5502548F550E54F8C
:10308A003EF54FED354EF54EEC354DF54DAF4CAEA8
:10309A004BAD4AAC49AB50AA4FA94EA84DD3122604
:1030AA00A140099080027410F07F002290802CE5E4
:1030BA004DF0A3E54EF0A3E54FF0A3E550F0908064
:0630CA00027440F0AF4665
:0130D00022DD
:10324E009081E3E0F54605460546054605460546EA
:10325E000546054605460546054690801CE0F5499F
:10326E00A3E0F54AA3E0F54BA3E0F54C9081E4E032
:10327E00F5460546054605460546054605460546F8
:10328E00054605460546908020E0F54DA3E0F54E37
:10329E00A3E0F54FA3E0F550E4F546E54FB54B0A34
:1032AE00E550B54C05C21F023399E54F540744E86B
:1032BE00F58385508263A20190600463A2017F0EA4
:1032CE00122BA6906004E0F547A3E0F54890600C41
:1032DE00E0FFF4604590667BE0FEEF6E706EA3E05B
:1032EE00FF90600DE06F706490667DE0FF90600E61
:1032FE00E06F705890667EE0FF90600FE06F704C4C
:10330E0090667FE0FF906010E06F7040906680E006
:10331E00FF906011E06F60048032D2D9906004E0BB
:10332E00702AA3E024F2F546E54F540744E8F583EE
:10333E00855082740E2582F582E43583F58363A26F
:10334E000190600463A201AF46122BA6AE47E4FCC7
:10335E00FDE5502548F550E54F3EF54FED354EF560
:10336E004EEC354DF54DAF4CAE4BAD4AAC49AB5076
:10337E00AA4FA94EA84DD31226A15006E54845479F
:10338E0070099080017410F07F0022908020E54D2E
:10339E00F0A3E54EF0A3E54FF0A3E550F0908001C9
:0533AE007440F0AF4681
:0133B30022F7
:0437F6008E4B8F4C1B
:1037FA00908000E030E5079065787401F022906BC4
:10380A000EE0FCA3E0FDA3E0FEA3E0F5528E518D8D
:10381A00508C4FE552FFE5515407FEE42FF54EEE6A
:10382A0034C0F54D854E82F5837423F0054EE54E7E
:10383A007002054D534DC7F582854D83740AF00514
:10384A004EE54E7002054D534DC790633E63A2018B
:10385A00854D83854E8263A2017F06122B4A740628
:10386A00254EF54EE4354DF54D854B83854C8263E7
:10387A00A201854D83854E8263A201122B2EE4FCA0
:10388A00FDFE906B0EE0F8A3E0F9A3E0FAA3E02FA7
:10389A00FFEE3AFEED39FDEC38FCEF2408FFE43E7A
:1038AA00FEE43DFDE43CFC906B0E1226B2906B0EDA
:1038BA00E0908040F0906B0FE0908041F0906B10A8
:1038CA00E0908042F0906B11E0908043F09080008D
:0338DA007420F067
:0138DD0022C8
:0A34F9008E4B8F4C8C4D8D4E8B4F87
:10350300908000E030E5079065787401F022906BBD
:103513000EE0FCA3E0FDA3E0FEA3E0F5558E548D81
:10352300538C52E555FFE5545407FEE42FF551EE55
:1035330034C0F550855182F5837423F00551E5516C
:10354300700205505350C7F582855083740AF00505
:1035530051E551700205505350C790633E63A20179
:1035630085508385518263A2017F06122B4A74061C
:103573002551F551E43550F550854B83854C8263D5
:10358300A20185508385518263A201122B2E8F568F
:10359300EF2551F551E43550F550E54F6017854D52
:1035A30083854E8263A20185508385518263A20184
:1035B300AF4F122B4AE5562408254FF54FFFE4FC85
:1035C300FDFEE5552FF555EE3554F554ED3553F520
:1035D30053EC3552F552908040E552F0A3E553F099
:1035E300A3E554F0A3E555F09080007420F0AF55A7
:0C35F300AE54AD53AC52906B0E1226B2D9
:0135FF0022A9
:0639BF008E478F488D4980
:1039C500908000E030E5079065787401F022906BF7
:1039D5000EE0FCA3E0FDA3E0FEA3E0F54F8E4E8DC7
:1039E5004D8C4CE54FFFE54E5407FEE42FF54BEEAD
:1039F50034C0F54A854B82F5837423F0054BE54BBE
:103A05007002054A534AC7F582854A83EBF0054B98
:103A1500E54B7002054A534AC790633E63A2018590
:103A25004A83854B8263A2017F06122B4A740625C1
:103A35004BF54BE4354AF54A85478385488263A2B1
:103A450001854A83854B8263A201AF49122B4A74D3
:103A5500082549F549FFE4FCFDFEE54F2FF54FEE3E
:103A6500354EF54EED354DF54DEC354CF54C90801C
:103A750040E54CF0A3E54DF0A3E54EF0A3E54FF08E
:103A85009080007420F0AF4FAE4EAD4DAC4C906BB6
:043A95000E1226B235
:013A9900220A
:024196008F5F39
:10419800908000E030E5079065787401F022906B1C
:1041A8000EE0FCA3E0FDA3E0FEA3E0F5638E628DC4
:1041B800618C60E563FFE5625407FEE42FFFEE348F
:1041C800C09062B463A201F5838F8263A201AF5FDE
:1041D800122B4AE4FCFDFEE563255FF563EE3562CC
:1041E800F562ED3561F561EC3560F560908040E58C
:1041F80060F0A3E561F0A3E562F0A3E563F09080C9
:10420800007420F0AF63AE62AD61AC60906B0E12CB
:0242180026B2CC
:01421A002281
:0638DE008E468F47AB058A
:1038E400908000E030E5079065787401F022906BD9
:1038F4000EE0FCA3E0FDA3E0FEA3E0F54D8E4C8DAD
:103904004B8C4AE54DFFE54C5407FEE42FF549EE98
:1039140034C0F548854982F5837423F00549E549A7
:10392400700205485348C7F582854883EBF0054982
:10393400E5497002054890633E63A201854883858A
:10394400498263A2017F06122B4A74062549F54970
:10395400E43548F5485348C7E54685498285488398
:10396400F00549E549700205485348C7F582854882
:1039740083E547F00549E549700205485348C7E522
:103984004D240AF54DE4354CF54CE4354BF54BE448
:10399400354AF54A908040E54AF0A3E54BF0A3E5AB
:1039A4004CF0A3E54DF09080007420F0AF4DAE4C88
:0A39B400AD4BAC4A906B0E1226B228
:0139BE0022E6
:0A49B000E4FEEEC39F50030E80F8F2
:0149BA0022DA
:103E4B00E4F546E5462401FFE433FE12469574364D
:103E5B002546F582E43463F583EFF00546E546C36A
:103E6B00943F40DFE4F546E546247FFFE433FE1242
:103E7B004695742D2546F582E43461F583EFF07495
:103E8B002D2546F582E43461F583E0FF6003B4FF32
:103E9B001D742D2546F582E43461F5837420F0748E
:103EAB002E2546F582E43461F583E4F0800905465E
:103EBB00E546C3948040B0E49061ACF0F546AF4664
:103ECB007E0012469574AD2546F582E43461F58388
:0B3EDB00EFF00546E546C394FE40E30F
:013EE60022B9
:10491300E4FDFCC3ED9FEC9E5015E4FBFA0BBB00DA
:0F492300010ABA01F8BB90F50DBD00010C80E44C
:014932002262
:0D4989004390014390025390FE5390FD2295
:0D4996005390FD5390FE4390024390012288
:0E497A005390FD439002E5905408FF5390FDCA
:01498800220C
:0D49A3005390FD4390014390025390FD227C
:0749C600AE071FEE70FA229C
:02482500AD07DD
:10482700E4FC5390FDEDA804088002C333D8FC30A4
:10483700E70543900180035390FE7F051249C64365
:0948470090020CBC08DC5390FD4A
:014850002245
:10487B00E4FF5390FD7E07439002E59030E00D740A
:10488B0001A806088002C333D8FC42075390FD1ED3
:08489B00C3EE6480948050DF3D
:0148A30022F2
:10485100AB05AA071249897FA012482512497AAFF0
:104861000212482512497AAF0312482512497A12D9
:0A48710049967F0A7E0012491322C7
:04469500AB07AA06BF
:10469900C3EB94FFEA9400400DE42BF58274773A5A
:1046A900F583E493FF221249897FA0124825124914
:1046B9007AAF0312482512497A1249897FA1124813
:0D46C9002512497A12487B1249A312499626
:0146D60022C1
:0247BE008B4B23
:1047C000A2AF9226C2AF85A24C53A2FE8E838F82E7
:1047D00005A28C838D827409122BD4E54B53A2FE63
:1047E00043A220122BD653A2DF854CA2A22692AF61
:0147F000FFC9
:0147F10022A5
:10493300A2AF9226C2AF8C838D82EF122BD443A2F7
:0C49430020122BD653A2DFA22692AFFF59
:01494F002245
:0248CB008F4616
:1048CD00A2AF9226C2AFE4F5838D827406122BD46B
:1048DD00E54643A220122BD653A2DFA22692AF7F2C
:0148ED0001C9
:0148EE0022A7
:0248EF008F46F2
:1048F100A2AF9226C2AFE4F5838D82740A122BD443
:10490100E54643A220122BD653A2DFA22692AF7F07
:0149110001A4
:014912002282
:1029FD00A907E7FFA805EF93C3966008403B74FC59
:102A0D002FFF80F00F08EF93C3966008402B74FBE7
:102A1D002FFF80E00F08EF93C3966008401B74FAF8
:102A2D002FFF80D00F08EF93D3966008400B74F9F9
:102A3D002FFF80C01F1F1F1F1FEF54FEF80303F74A
:102A4D00E893FC08E893FD08E893FE08E893FF225D
:102A5D0009E993C39D6008402974FB29F980F109A8
:102A6D00E993C39E6008401A74FA29F980E209E9D6
:102A7D0093D39F6008400B74F929F980D319191964
:102A8D001919E9C313C313FF22740093F8ECC3980B
:102A9D004024701F740193F8EDC39840197014749D
:0E2AAD000293F8EEC398400E7009740393F87C
:102ABB00EFC39840037F00227F0122EDF8E6F00878
:102ACB00A3DFFA22EDF8E0F608A3DFFA22E0A36316
:102ADB00A201F0A363A201DFF475A2002263A2019D
:102AEB00F0A363A20122E0A363A201F0A363A201FE
:102AFB00E0A363A201F0A363A201E463A201F0A32C
:102B0B0063A201DFE175A20022E0A363A2016DFEC7
:102B1B00936CFDEE058393FC158363A201DFEA75CD
:102B2B00A200227F00E493A363A201F00F600CA329
:102B3B00E583C2E3F58363A20180EA75A20022E07C
:102B4B00A363A201F0A3E583C2E3F58363A201DFD4
:102B5B00EE75A20022E0A363A201F0A3E583C2E419
:102B6B00D2E3F58363A201DFEC75A20022E0A3633D
:102B7B00A201F0A3E58344F8C2E5F58363A201DF6C
:102B8B00EC75A20022E583C2E3F583E0A363A20107
:102B9B00F0A363A201DFEE75A20022E583C2E4D2AB
:0A2BAB00E3F583E0A363A201F0A3A9
:102BB50063A201DFEC75A20022E58344F8F583E00A
:102BC500A363A201F0A363A201DFEE75A20022F9BF
:102BD50022C002C004C00612FFF0D006D004D00205
:012BE50022CD
:10001E00BF360BD209E4F526F527F542F543BF3777
:04002E0002C20922DF
:1044E100C2A9438902906B09E0FFF58C8F8A75D9C7
:1044F1000475DA4875DB3175DC4975DD4975DE31E6
:10450100E4F5E9F5F9F5EBF5FB906B07E06016755D
:10451100EC1075ED10E4F5FCF5FD753E08753C10E9
:10452100753D01801375EC8075ED80E4F5FCF5FDBA
:0E453100753E80F53C753D10E4F5EEF5FE227A
:10471800E4FEAF8CEFFD906B08E07003A3E06D60E2
:10472800051244E17E01E5D920E2057E021244E14A
:10473800E58920E1051244E17E03D28C75D84075E5
:08474800B740D2AED2AFAF06BC
:014750002246
:030033000230D1C7
:0B30D100C0E0C083C082C0D075D008F2
:1030DC00C2AF30DC56C3E5EC95EEC3953E5012E51D
:1030EC003D25ECF5EC30D70405FC801685FCFC8006
:1030FC0011C3E5EC953DF5EC30D70415FC80038548
:10310C00FCFC300924852782852683E590F0052771
:10311C00E52770020526F582852683E5EEF0052766
:10312C00E5277002052653260FC2DC30D929300959
:10313C0024852782852683E590F00527E5277002F4
:10314C000526F582852683E5EBF00527E527700239
:10315C00052653260FC2D930DA69E53C700405FC0C
:10316C008010E53C25ECF5EC30D70405FC8003859C
:10317C00FCFC300A4CE5285480FFE52825E0F528B6
:10318C003097020528200803632801302F19E52801
:10319C0054C06544702BEF7028753F08F53A8528AC
:1031AC002BF528C22F801A053FE53F5407701253A8
:1031BC003F3FE53F131313541F242AF8A628752804
:1031CC0000C2DA30DB71E53C700405FD8010E53C93
:1031DC0025EDF5ED30D70405FD800385FDFDE540BB
:1031EC00653B6029E53B54077013E53B13131354FF
:1031FC001F2432F8E6F5292007036329FFE529335C
:10320C009296E52925E0F529053B533B3FB29230D8
:10321C000923852782852683E590F00527E527700D
:10322C00020526F582852683E4F00527E527700242
:09323C00052653260FC2DBD2AFB8
:09324500D0D0D082D083D0E03259
:101DDB004241554400575F4D4F44454D00494E56C7
:101DEB005F52454300494E565F5452414E53004992
:101DFB004E565F414C4C004C495354454E004E5F80
:101E0B004B50005052494F520047525F54495400B7
:101E1B00575F414E535700003E2A2C312CCFE0F038
:101E2B00E0ECE5F2F0FB20F1E8EDF5F0EEEDEDEE98
:101E3B00E3EE20EFEEF0F2E00A003E4C2C423031A4
:101E4B002C256C752CD1EAEEF0EEF1F2FC20EEE1D4
:101E5B00ECE5EDE02C35302C3130302C3230302CA1
:101E6B003330302C3630302C313230302C32343061
:101E7B00302C343830300A003E422C4731302C2580
:101E8B0062752CC8EDE2E5F0F1E8FF20EDE020EF04
:101E9B00F0E8B8ECE50A003E422C4731312C2562C4
:101EAB00752CC8EDE2E5F0F1E8FF20EDE020EFE561
:101EBB00F0E5E4E0F7E50A003E422C4730322C25F2
:101ECB0062752CD3EFF0E0E2EBE5EDE8E520EFEE09
:101EDB00F2EEEAEEEC2020285254532D43545329B2
:101EEB000A003E532C4730332C256C752CC7E0E48D
:101EFB00E5F0E6EAE020F1F2E0F0F2E020EFE5F0C9
:101F0B00E5E4E0F7E828ECF1290A003E532C4730D2
:101F1B00332C256C752C202AE7E0E4E5F0E6EAE0AB
:101F2B0020F1F2E0F0F2E020EFE5F0E5E4E0F7E895
:101F3B0028ECF1290A003E2A2C312CC0E4E0EFF208
:101F4B00E5F020F1E8EDF5F0EEEDEDEEE3EE20EA55
:101F5B00E0EDE0EBE02E20CFF0EEF2EEEAEEEB2040
:101F6B00CAEEECEFE0F120D2CC312E310A003E422A
:101F7B002C4B30342C2562752CD0E5E6E8EC20EFA9
:101F8B00F0EEF1EBF3F8EAE820EAE0EDE0EBE0202D
:101F9B00F1E2FFE7E80A003E532C4B30312C25735E
:101FAB002CD1EFE8F1EEEA20CACF0A003E532C4BBE
:101FBB0030322C25732CCAEEEB2DE2EE20E3F0F33E
:101FCB00EFEF20D2C8D20A003E532C4B30332C25D6
:101FDB00732CCFF0E8EEF0E8F2E5F220CED220EA57
:101FEB0020C7C3D2C8D20A003E532C4732302C250F
:101FFB006C752CC2F0E5ECFF20EEE6E8E4E0EDE8D2
:10200B00FF20EEF2E2E5F2E028ECF1290A003C2198
:10201B00003C4230313D003C4731303D003C4731C4
:10202B00313D003C4730323D003C4730333D003CB6
:10203B004732303D003C4B30343D003C4B30313D62
:10204B00003C4B30323D003C4B30333D000ACFEE71
:10205B00EFFBF2EAE020EEF2EFF0E0E2EAE820F14B
:10206B00EBE8F8EAEEEC20E4EBE8EDEDEEE3EE2046
:10207B00EFE0EAE5F2E021000ACEF2EFF0E0E2EA6F
:10208B00E020D2D30A000ACEF2EFF0E0E2EAE02041
:10209B00E7E0EFF0EEF1E020EEF220F1E5F0E2E523
:1020AB00F0E00A000A435243206572726F722100FE
:1020BB000ACFF0E8B8EC20E8EDF4EEF0ECE0F6E84F
:1020CB00E8000AD7F3E6EEE920CACF21000AC6E4FE
:1020DB00E0EB20E8EDF4F320E020F2F3F220F7F24E
:1020EB00EE2DF2EE20EDE520F2EE2E2E2E000ACA9A
:1020FB00E2E8F2E0EDF6E8FF20D2D321000ACDE5CD
:10210B00F220E8EDF4EEF0ECE0F6E8E821000ACF7F
:10211B00F0E8B8EC20E7E0EFF0EEF1E0000ACDE0FC
:10212B00F7E0EBEE20EFF0E8B8ECE0000AC8F1F2D4
:10213B00E5EAEBEE20E2F0E5ECFF20EEE6E8E4E08A
:10214B00EDE8FF20EEF2E2E5F2E0000AC7E0EFF087
:10215B00EEF120E3F0F3EFEFFB20D2C8D22000200A
:10216B00EEF220CACF20000A000ACEF2EFF0E0E236
:10217B00EAE020CED220EDE020CACF2000202020A4
:10218B00CFEEE2F2EEF020EAEEECE0EDE4FB0A003B
:10219B00FF1DDBFF1DE0FF1DE8FF1DF0FF1DFAFF1C
:1021AB001E02FF1E09FF1E0EFF1E14FF1E1BFF1E2D
:0121BB002201
:103C430052668D000000000000000000000000002C
:103C5300000000000060A06A60000500020000058B
:103C6300000200000500020000050002000005003C
:103C7300020000050002000005000200000500022A
:103C8300000005000200000500020000050002001C
:103C9300000500020000050002000005000200000C
:103CA30005000200000500020000050002000005F7
:103CB30000020000050002000005000200000500EC
:103CC30002000005000200000500020000050002DA
:103CD30000000500020000050002000005000200CC
:103CE30000050002000005000200000500020000BC
:093CF300050002000005000200BA
:0100320022AB
:0245F5008F51E4
:1045F700906B05E0FF04F074B82FF582E43467F59B
:10460700837420F0E4FFEFC39D503BE55175F00341
:10461700A4249BF582E43421F583E493FB7401938E
:10462700FA740293F98F82758300122531FE906B1D
:1046370005E024B8F582E43467F583EEF00F906B5C
:0646470005E004F080C054
:01464D00224A
:1048A400742D2FF582E43461F583E0FE64206016F4
:1048B400906B05E0FD04F074B82DF582E43467F5DF
:0648C40083EEF00F80DA24
:0148CA0022CB
:10195600E4906B05F0F548E54875F003A4249BF583
:1019660082E43421F583E493FB740193FA740293C1
:10197600F91225187003021DDAE4F54AF54BF5490C
:10198600742D2549F582E43461F583E0FF70030286
:101996001DD5E54875F003A4249BF582E43421F5B2
:1019A60083E493FB740193FA740293F9854A827572
:1019B6008300122531FEEFB50608754B01054A0274
:1019C6001DD0E54B7003021DD0EE6003021DCBADAA
:1019D6004AAF481245F5E548B40A004003021DD552
:1019E6009019EDF8282873021A0B021AA9021ADFB9
:1019F600021AE4021AE9021AF0021AF5021BD202CE
:101A06001CB5021D98AF491248A4742D2549F9E466
:101A16003461FA7B01C0031B8B5475550075560063
:101A2600E4F557D003122DA68F508E4F8D4E8C4D58
:101A3600E4FFFEFDFCAB50AA4FA94EA84DC31226EB
:101A4600A16022AB50AA4FA94EA84DE47F207E1C70
:101A5600FDFC122601122693906B08EEF0A3EFF020
:101A6600E4906B07F0E47FB07E04FDFCAB50AA4F18
:101A7600A94EA84DD31226A15003021DD5906B077F
:101A86007401F0AB50AA4FA94EA84D7F007EC2FD4F
:101A96007C00122601122693906B08EEF0A3EFF05D
:101AA600021DD5AF491248A4D20C742D2549F9E47C
:101AB6003461FA7B01C0031B8B54755500755600C3
:101AC600E4F557D003122DA68F508E4F8D4E8C4DB8
:101AD60090671FE550F0021DD5D208021DD5D2072A
:101AE600021DD5D208D207021DD5D213021DD5AFCD
:101AF600491248A4E4F54C742D2549F9E43461FAF9
:101B06007B01C0031B8B54755500755600E4F557D1
:101B1600D003122DA68F508E4F8D4E8C4DE54C75F1
:101B2600F005A42460F9746A35F0FA7B01906B0124
:101B3600EBF0A3EAF0A3E9F0E550122591742D2508
:101B460049F582E43461F583E0FF642060047E0198
:101B560080027E00EF60047F0180027F00EF5E70EE
:101B660003021DD50549742D2549F582E43461F536
:101B760083E0B42CC8054CE54CC394204003021DF9
:101B8600D50549742D2549F9E43461FA7B01C00372
:101B96001B8B54755500755600E4F557D003122D6E
:101BA600A68F508E4F8D4E8C4DE54C75F005A424B6
:101BB60060F9746A35F0FA7B01906B01EBF0A3EAE9
:101BC600F0A3E9F0E550122591021B43AF491248F4
:101BD600A4E4F54C742D2549F9E43461FA7B01C07F
:101BE600031B8B54755500755600E4F557D0031248
:101BF6002DA68F508E4F8D4E8C4DE54C75F005A45D
:101C06002460F9746A35F0FA7B01906B01EBF0A35E
:101C1600EAF0A3E9F0900001E5501225A3742D2502
:101C260049F582E43461F583E0FF642060047E01B7
:101C360080027E00EF60047F0180027F00EF5E700D
:101C460003021DD50549742D2549F582E43461F555
:101C560083E0B42CC8054CE54CC394204003021D18
:101C6600D50549742D2549F9E43461FA7B01C00391
:101C76001B8B54755500755600E4F557D003122D8D
:101C8600A68F508E4F8D4E8C4DE54C75F005A424D5
:101C960060F9746A35F0FA7B01906B01EBF0A3EA08
:101CA600F0A3E9F0900001E5501225A3021C23AF32
:101CB600491248A4E4F54C742D2549F9E43461FA37
:101CC6007B01C0031B8B54755500755600E4F55710
:101CD600D003122DA68F508E4F8D4E8C4DE54C7530
:101CE600F005A42460F9746A35F0FA7B01906B0163
:101CF600EBF0A3EAF0A3E9F0900003E5501225A368
:101D0600742D2549F582E43461F583E0FF64206093
:101D1600047E0180027E00EF60047F0180027F0066
:101D2600EF5E7003021DD50549742D2549F582E441
:101D36003461F583E0B42CC8054CE54CC3942040CF
:101D460003021DD50549742D2549F9E43461FA7B52
:101D560001C0031B8B54755500755600E4F557D02A
:101D660003122DA68F508E4F8D4E8C4DE54C75F07F
:101D760005A42460F9746A35F0FA7B01906B01EBD7
:101D8600F0A3EAF0A3E9F0900003E5501225A302C0
:101D96001D06AF491248A4742D2549F9E43461FAA9
:101DA6007B01C0031B8B54755500755600E4F5572F
:101DB600D003122DA68F508E4F8D4E8C4D9067B747
:101DC600E550F0800AE4F54BF54A05490219860507
:041DD6004802195D49
:011DDA0022E6
:1033B4007BFF7A1E792312221E906B07E0602FA3F5
:1033C400E0FEA3E0FFC3E49FFFE49EFEAB07FAE444
:1033D400F9F8FF7EC27D01FC1226018F518E508DBB
:1033E4004F8C4E7BFF7A1E794512221E802F906BE4
:1033F40008E0FEA3E0FFC3E49FFFE49EFEAB07FAF0
:10340400E4F9F87F207E1CFDFC1226018F518E50BA
:103414008D4F8C4E7BFF7A1E794512221E7BFF7ADC
:103424001E7983A208E433F54E12221E7BFF7A1E16
:1034340079A2A207E433F54E12221E7BFF7A1E798D
:10344400C3A20CE433F54E12221E300C1F7BFF7A0C
:103454001E79ED90671FE075F00AA4FFAEF0E48FCB
:10346400518E50F54FF54E12221E801D7BFF7A1FA0
:10347400791690671FE075F00AA4FFAEF0E48F514F
:103484008E50F54FF54E12221E7BFF7A1F794112A2
:10349400221E7BFF7A1F7979A213E433F54E1222A0
:1034A4001E754E01754F677550207BFF7A1F79A2F8
:1034B40012221E754E01754F687550B87BFF7A1F36
:1034C40079B712221E754E01754F6675509F7BFFAA
:1034D4007A1F79D312221E7BFF7A1F79F39067B784
:1034E400E075F00AA4FFAEF0E48F518E50F54FF56D
:0534F4004E12221E2211
:02429F008D4848
:1042A100AA06A907754B018A4C894DE4F5491249C3
:1042B100508F4AE54A643C6030E54A642C602AAB81
:1042C1004BAA4CA94DE54A1225917401254DF54D96
:1042D100E4354CF54C05491249508F4AE54A643C96
:1042E1006007E549C3954840D6E5497016AB4BAA2E
:1042F1004CA94D74201225917401254DF54DE435DD
:104301004CF54CE549B5480C74FF254DF54D74FF4E
:0E431100354CF54CAB4BAA4CA94DE41225914E
:01431F00227B
:1027DE007E207F19124111EF4E70037F01227E2061
:1027EE007F1C124111EF4E700302288512453F9057
:1027FE006B1B1226B2E4FFFEFDFC906B1BE0F8A3F0
:10280E00E0F9A3E0FAA3E0FBC31226A16025906BCA
:10281E001BE0F8A3E0A3E0A3E0E47F207E1CFDFC18
:10282E00122601122693906B08EEF0A3EFF0E490BF
:10283E006B07F0E47FB07E04FDFC906B1BE0F8A309
:10284E00E0F9A3E0FAA3E0FBD31226A14038906B87
:10285E00077401F0906B1BE0F8A3E0A3E0A3E07F08
:10286E00007EC27D017C00122601122693906B0819
:10287E00EEF0A3EFF0800F906B0874FFF0A374B826
:10288E00F0E4906B07F07E207F22124111EF4E6034
:10289E000C124950EF24D024FF92088002C2087E09
:1028AE00207F28124111EF4E600C124950EF24D0B8
:1028BE0024FF92078002C2077E207F2E124111EF65
:1028CE004E600C124950EF24D024FF920C8002C2AD
:1028DE000C7E207F34124111EF4E601312453FE4FF
:1028EE007B0AFAF9F812260190671FEFF08005E4D3
:1028FE0090671FF07E207F3A124111EF4E60111249
:10290E00453FE47B0AFAF9F81226019067B7EFF01B
:10291E009067B7E07003740AF07E207F4012411179
:10292E00EF4E600C124950EF24D024FF9213800218
:10293E00C213E4906B1AF07E207F46124111EF4EC7
:10294E00600B7E677F207D8012429F8023906B1AE2
:10295E00E0FF04F074202FF582E43467F5837420D1
:10296E00F0906B1AE02420F582E43467F583E4F0EE
:10297E00E4906B1AF07E207F4C124111EF4E600BEB
:10298E007E687FB87D8012429F8023906B1AE0FF95
:10299E0004F074B82FF582E43468F5837420F09057
:1029AE006B1AE024B8F582E43468F583E4F0E49021
:1029BE006B1AF07E207F52124111EF4E600B7E6635
:1029CE007F9F7D8012429F8023906B1AE0FF04F060
:1029DE00749F2FF582E43466F5837420F0906B1AA1
:0E29EE00E0249FF582E43466F583E4F07F0078
:0129FC0022B8
:1047890030122FE4906475F0A3E56FF090667AE03B
:10479900906477F0A37405F0906960E0543FF0638A
:1047A900A20190647963A201AF6F122AD8C2127F65
:0547B90001227F002237
:102BE600906B0874FFF0A374B8F0E4906B07F09054
:102BF6006B05F0C2101227DEEF6006121956022D81
:102C0600A2E4F547F54674202546F582E43467F5D7
:102C160083E0FF6070E547C394205069EFB4200459
:102C2600054680E2E54775F005A42460F9746A3527
:102C3600F0FA906B017401F0A3EAF0A3E9F07420B6
:102C46002546F9E43467FA7B01C0031B8B5475559E
:102C560000755600E4F557D003122DA6906B01E0DF
:102C6600FBA3E0FAA3E0F9EF1225910547742025AE
:102C760046F582E43467F583E0FF64206088EF6000
:102C860085054680E8E5477005D210022DA2E4F5D9
:102C960047F54674B82546F582E43468F583E0FFC7
:102CA6006073E547C39420506CEFB420040546805A
:102CB600E2E54775F005A42460F9746A35F0FA90E8
:102CC6006B017401F0A3EAF0A3E9F074B82546F9A4
:102CD600E43468FA7B01C0031B8B547555007556A6
:102CE60000E4F557D003122DA6906B01E0FBA3E09C
:102CF600FAA3E0F9900003EF1225A3054774B8255F
:102D060046F582E43468F583E0FF64206085EF6071
:102D160082054680E8E4F547F546749F2546F58228
:102D2600E43466F583E0FF6073E547C39420506C96
:102D3600EFB42004054680E2E54775F005A424605B
:102D4600F9746A35F0FA906B017401F0A3EAF0A306
:102D5600E9F0749F2546F9E43466FA7B01C0031B4B
:102D66008B54755500755600E4F557D003122DA601
:102D7600906B01E0FBA3E0FAA3E0F9900001EF12EB
:102D860025A30547749F2546F582E43466F583E05E
:0F2D9600FF64206085EF6082054680E81244E10B
:012DA500220B
:1047F2007544C0C209C206E4F528C212C20FC20142
:10480200D211F53AF53FF5749067B6F030130D7595
:104812006703D22FA3E09067B6F08003E4F5671236
:0348220047182212
:10441400D227E4FEE56C25E0F56CEF30E708436C49
:1044240001A227B39227056EE56EB40816856B8248
:10443400856A83E56CF0056BE56B7002056A0570AF
:10444400E4F56EEF25E0FF0EBE08C9E56C25E0F546
:104454006CA226302701B35003436C01056EE56E50
:10446400B40816856B82856A83E56CF0056BE56B91
:094474007002056A0570E4F56EA2
:01447D00221C
:02370400AB0711
:10370600E4FD200038906B00E0FF30E10A6402F02F
:10371600906B04E06429F0906B00E0FF25E0F090E8
:103726006B04E0FE30E707906B00E04401F0EE2505
:10373600E0906B04F0EB30E704E04401F0056EE541
:103746006E24F8601E1460418000EB30E70A437572
:1037560001A204B3920480035375FEE57525E0F5D6
:1037660075807DEB30E70A437501A204B3920480AD
:10377600035375FE856982856883E575F00569E5FD
:103786006970020568056F8057300526D20E300D28
:103796001E906B00E0FF30E10A6402F0906B04E0DB
:1037A6006429F0906B04E0FF906B00E04FFF227FEE
:1037B6000022300413EB20E720D205E575B420047F
:1037C600D20D8015C20D8011EB30E70DD205E575DF
:1037D600B42004D20D8002C20DC200D204E4F56EFC
:0F37E600EB25E0FB0DED640860030237087F0060
:0137F50022B1
:0246D700AD072D
:1046D900E4F5707B387A69756A69756BE08B828A53
:1046E90083E044C0F0E4F56EFCECC39D50138B826B
:1046F9008A83E0FFC2261244140BBB00010A0C8016
:0E470900E8D226E4FF124414756A69756BE06D
:01471700227F
:023DAD008F463F
:103DAF00300103023E4A74FC2546F54613131354A3
:103DBF001FFF2546FFE433CF2402CF3400FEC3EFAD
:103DCF009414EE64809480401130230B7E207F5832
:103DDF00E4FBFDFC1234F9D21122754701856A48C4
:103DEF00856B49AD70E4F5707B797A63756A677599
:103DFF006BA18B828A83E044C0F0AC6EE4F56EF960
:103E0F00E9C3954650138B828A83E0FFC226124482
:103E1F00140BBB00010A0980E7D226E4FF124414F9
:103E2F00D2019067B5E570F08D7085486A85496B52
:0B3E3F007571017572677573A18C6EC0
:013E4A002255
:103A9A00E4FF0F2405F582E43461F5837405F00F21
:103AAA0074052401F582E43461F583E4F075460176
:103ABA00754766754892FEAB46E5481548AA4770B1
:103ACA00021547F9122518FDAC070F74052CF5826B
:103ADA00E43461F583EDF00EBE04DC7546017547EA
:103AEA0066754896E4FEAB46E5481548AA47700253
:103AFA001547F9122518FDAC070F74052CF582E459
:103B0A003461F583EDF00EBE04DC75460175476637
:103B1A0075489AE4FEAB46E5481548AA477002156F
:103B2A0047F9122518FDAC070F74052CF582E43409
:103B3A0061F583EDF00EBE04DC75460175476675C6
:103B4A00489EE4FEAB46E5481548AA477002154769
:103B5A00F9122518FDAC070F74052CF582E43461BF
:083B6A00F583EDF00EBE04DC52
:013B72002230
:100ED70030092DC3E5279543FFE5269542FED3EF5D
:100EE7009440EE940040197B087D40AF43AE421218
:100EF70039BFE5432440FFE43542540FF5428F43A1
:100F070020190302149730180AC2189067B6E060D8
:100F17000214F0E567B40700501C900F28F8282842
:100F270073020F41020FF2020FF20210E3021307DE
:100F37000210E3021472E4F5672230131075670399
:100F4700D22F9067B7E09067B6F0D20A222001034C
:100F5700020FEE9067B5E0F570C201D214E4F546D2
:100F6700E546C395705026AB71AA72A9731225186E
:100F7700FF74382546F582E43469F583EFF0740190
:100F87002573F573E43572F572054680D3756A6982
:100F9700756B38856A65856B66857064856B828538
:100FA7006A83A3E0547FFF64706003BF381F7567CF
:100FB700019067A07406F0D2032023030214977EE2
:100FC700207F83AB70AD6BAC6A1234F92230230DEE
:100FD7007E207F91AB70AD6BAC6A1234F9756701F7
:100FE7009067A07403F02275670422200F03021094
:100FF7009BE540653B6047E54024085438FFE53BE7
:1010070054386F60047E0180027E00E57060047DC5
:101017000180027D00EE5D7003021497856B828567
:101027006A83E0FEE540131313541F2432F8A60623
:101037008F40056BE56B7002056A157080B9906784
:10104700A0E06406603F301404D211C21490669386
:10105700E0FCA3E0FDA3E0FEA3E0FFE4FAF9F8EF6C
:101067002401FFEA3EFEE93DFDE83CFC9066931251
:1010770026B2D20AE4F528D22FD2B19067B7E09012
:1010870067B6F080069067B67441F0C20F9067A00C
:10109700E0F5672230B10B300C0890671FE09067CE
:1010A700B6F0C2B1300C0C30B0099067B6E06003FF
:1010B700021497856B82856A83E0FFE5401313135B
:1010C700541F2432F8A607E54024085438F5400594
:1010D7006BE56B7002056A1570D20F2220060302BA
:1010E7001299E53F5438653A7003021497E53A249C
:1010F700085438F53A131313541F242AF8E6F56DEC
:1011070020050FFF1237048F46E56FD3948040D236
:101117008025200D030211D4E567640360030211E3
:10112700D4AF6D1237048F46300EB7C20EC206C257
:1011370005C20AE5466039C21230230D7E207FAF13
:101147007C697D60AB6F1234F9906697E0FCA3E091
:10115700FDA3E0FEA3E0FFE4FAF9F8EF2401FFEABC
:101167003EFEE93DFDE83CFC9066971226B28059A9
:10117700906938E0FF906960E06F703D156F156FFB
:10118700D21230230D7E207FBB7C697D60AB6F124E
:1011970034F990668FE0FCA3E0FDA3E0FEA3E0FF37
:1011A700E4FAF9F8EF2401FFEA3EFEE93DFDE83CE9
:1011B700FC90668F1226B2801030230D7E207FCDE3
:1011C7007C697D60AB6F1234F9E4F56722E567B49B
:1011D700031630230D7E207FD87C697D60AB6F12AC
:1011E70034F9E4F56702129030031CC203D21215DA
:1011F7006F30230D7E207FF97C697D60AB6F1234E1
:10120700F9E4F567021290906938E0FF906960E0B1
:101217006F601530230D7E207FCD7C697D60AB6FBD
:101227001234F9E4F5678061906939E0FF906961EC
:10123700E0B5071530230D7E217F087C697D60AB03
:101247006F1234F9E4F567804030230F7E217F1950
:101257007C697D60E56F14FB1234F9301305E4F502
:10126700678026906960E0906938F0906961E09046
:101277006939F0906962E090693AF07F031246D7C6
:101287007567019067A07403F0C20EC206C205C25B
:101297000A22202F2C30230B7E217F28E4FBFDFC24
:1012A7001234F9E49067B6F0D206F56F906B04F04C
:1012B700906B00F0D204F56ED200756869756960AD
:1012C700229067B6E0600302149730230A7E217FDD
:1012D70037FBFDFC1234F990669BE0FCA3E0FDA30D
:1012E700E0FEA3E0FFE4FAF9F8EF2401FFEA3EFE8F
:1012F700E93DFDE83CFC90669B1226B2E4F56722C7
:10130700301004E4F567220574E574C394204003A4
:10131700E4F574E57475F005A42460F9746A35F092
:10132700FA7B01906B01EBF0A3EAF0A3E9F0122539
:1013370018FF700302146B906B01E0FBA3E0FAA3A4
:10134700E0F9900002740112255E90000112253128
:10135700FE900002122531C39E5003021419906BB0
:1013670001E0FBA3E0FAA3E0F9900002E41225A351
:10137700900004740112255E900003122531FE903F
:101387000004122531D39E4013906B01E0FBA3E0CC
:10139700FAA3E0F990000474011225A3906B01E011
:1013A700FBA3E0FAA3E0F9906938EFF0A37410F01B
:1013B70090000412253190693AF09067A07403F009
:1013C700FF1246D72023030214677E217F56906BB6
:1013D70001E0A3E0FAA3E02404F9E43AFCAD017BC1
:1013E700011234F97F1E1249B07E217F6A906B018A
:1013F700E0A3E0FAA3E0AC02FD7B011234F97F1E03
:101407001249B07E217F727C697DE0AB701234F99E
:10141700804E906B01E0FBA3E0FAA3E0F9122518D8
:10142700906938F0A37450F0E4A3F09067A07405B6
:10143700F07F031246D73023277E217F74906B01FC
:10144700E0A3E0FAA3E0AC02FD7B011234F97F1EB2
:101457001249B07E217F727C697DE0AB701234F94E
:10146700756701227574FFE4F567229067B6E0702F
:101477001F30230A7E217F88FBFDFC1234F9756734
:10148700019067A07405F085656A85666B85647051
:011497002232
:0B49BB00301105C2117F01227F002295
:0349CD00C2AE2255
:103F830002090EE493A3F8E493A34003F68001F23D
:103F930008DFF48029E493A3F85407240CC8C3333F
:103FA300C4540F4420C8834004F456800146F6DF0E
:103FB300E4800B0102040810204080903C3DE47E25
:103FC300019360BCA3FF543F30E509541FFEE49303
:103FD300A360010ECF54C025E060A840B8E493A3CA
:103FE300FAE493A3F8E493A3C8C582C8CAC583CAF5
:103FF300F0A3C8C582C8CAC583CADFE9DEE780BEAD
:013CFC0000C7
:10251800BB010689828A83E0225002E722BBFE02C1
:09252800E32289828A83E49322F4
:10253100BB010CE58229F582E5833AF583E022505F
:1025410006E92582F8E622BBFE06E92582F8E222A9
:0D255100E58229F582E5833AF583E49322C3
:10255E00BB010FF8E58229F582E5833AF583E02881
:10256E00F0225009C58229F8E58226F622BBFE0923
:10257E00C58229F8E22582F222F8EA2583F583E95D
:03258E009328226D
:10259100BB010689828A83F0225002F722BBFE0129
:0225A100F32223
:1025A300F8BB010DE58229F582E5833AF583E8F06E
:1025B300225006E92582C8F622BBFE05E92582C81A
:0225C300F22202
:1025C50075F008758200EF2FFFEE33FECD33CDCCCD
:1025D50033CCC58233C5829BED9AEC99E582984050
:1025E5000CF582EE9BFEED9AFDEC99FC0FD5F0D62D
:1025F500E4CEFBE4CDFAE4CCF9A88222B800C1B957
:102605000059BA002DEC8BF084CFCECDFCE5F0CB94
:10261500F97818EF2FFFEE33FEED33FDEC33FCEBCD
:1026250033FB10D703994004EB99FB0FD8E5E4F988
:10263500FA227818EF2FFFEE33FEED33FDEC33FC75
:10264500C933C910D7059BE99A4007EC9BFCE99A69
:10265500F90FD8E0E4C9FAE4CCFB2275F010EF2FAE
:10266500FFEE33FEED33FDCC33CCC833C810D707AE
:102675009BEC9AE899400AED9BFDEC9AFCE899F8E9
:0E2685000FD5F0DAE4CDFBE4CCFAE4C8F9227C
:0E269300C3E49FFFE49EFEE49DFDE49CFC2258
:1026A100EB9FF5F0EA9E42F0E99D42F0E89C45F08F
:0126B1002206
:0C26B200ECF0A3EDF0A3EEF0A3EFF0229B
:1026BE00A8828583F0D083D0821226D51226D51219
:1026CE0026D51226D5E473E493A3C583C5F0C5833E
:1026DE00C8C582C8F0A3C583C5F0C583C8C582C866
:0126EE0022C9
:1021BC00E55A244EF8E6055A22784B302D02784E1B
:1021CC00E475F00112273E0225182026EB7F2ED253
:1021DC00268018EF540F2490D43440D4FF302A0BAF
:1021EC00EF24BFB41A0050032461FFE55B600215B5
:1021FC005B055EE55E7002055D302D0D784BE47578
:10220C00F00112273EEF02259102464E7403D22DA7
:10221C008003E4C22DF55A8B4B8A4C894DE4F55B57
:10222C00F55DF55EE55B60077F201221F780F575A3
:10223C005CFFC227C226C228C229C22BC22CC22EC6
:10224C001221C5FF700D302D057F00122208AF5EE4
:10225C00AE5D22B4255FC2D5C22A1221C5FF24D09F
:10226C00B40A00501A75F00A785B30D50508B6FF31
:10227C000106C6A426F620D5047002D22980D924E2
:10228C00CFB41A00EF5004C2E5D22A022408D22798
:10229C0080C6D22680C0D22880BCD2D580BAD22BA0
:1022AC0080B47F201221F72028077401B55B004011
:1022BC00F11221BCFF1221F7022230D22ED22C8037
:1022CC00951221BCFB1221BCFA1221BCF94A4B70AD
:1022DC000679D97A247BFF20282EE55B602A7E00C4
:1022EC008E8275830012253160060EEE655C70F0EF
:1022FC00C2D5EBC0E0EAC0E0E9C0E0EE12244FD05A
:10230C00E0F9D0E0FAD0E0FB122518FF60AAEBC090
:10231C00E0EAC0E0E9C0E01221F7D0E02401F9D0F6
:10232C00E03400FAD0E0FBE55C0460DCD55CD980DD
:10233C00877BFF7A24794BD228809C791080027994
:10234C0008C22CC22E8008D2D5790A8004790AC220
:10235C00D5E55C047002F55CE4FAFDFEFF1221BCCD
:10236C00FC7B082027131221BCFD7B1030260A129F
:10237C0021BCFE1221BCFF7B20EC3382D592D550C0
:10238C0013C3E43026069FFFE49EFEE42027039D42
:10239C00FDE49CFCE4CBF8C227EC700CCFCECDCC8A
:1023AC00E824F8F870F38017C3EF33FFEE33FEED3B
:1023BC0033FDEC33FCEB33FB994002FB0FD8E9EB1C
:1023CC00302705F8D0E0C448B227C0E00AEC4D4EE7
:1023DC004F78207B0070C2EAB55C0040BCC0E012B4
:1023EC002451D0F0D0E0202704C4C0E0C4B227C0F0
:1023FC00F01221E0D0F0D5F0EB02223012279D2212
:10240C00CD53234758229E4C229A42234B4F2353A1
:0F241C004423534922B343235955233D46233DBF
:10242B0045233D4724F95022A22D22A62E22C92B4B
:10243B0022AA2322C72024E22A226248000022C1BA
:10244B003F3F3F00790AA2D5202914302B09B91040
:10245B00020404B9080104A2D5202C025001042067
:10246B0028689228B55B005034C0E07F20302919D2
:10247B007F30A228722C722B500F1224A8C228C2B4
:10248B002CC22BC22E7F30800F302B03E9C0E01201
:10249B0021F7302B03D0E0F9D0E0B55BCC302B1714
:1024AB007F30B9100C1221F77F58302A077F7880C4
:1024BB0003B908031221F73028057F2D0221F77F7E
:1024CB0020202EF87F2B202CF322922880CF286EF1
:1024DB00756C6C2900D2271221BC3027F8C22778E3
:1024EB005B30D50108F60222622D50434958122168
:1024FB00BC2403B405004001E49024F4931221E8BA
:0D250B00743A1221E8D229755B04022347BF
:102DA6008B518A528953E4F55DF55CF55BF55AF56E
:102DB60058F559E555455645546012EBC0E0EAC052
:102DC600E0E9C0E0AB54AA55A95612274EAB51050F
:102DD60053E553AA527002055214F9122518F55EEE
:102DE600C394094007E55ED3940D40E1E55E642097
:102DF60060DBE55EB42D054359038016E55EB42B12
:102E060005435901800C74FF2553F55374FF355261
:102E1600F552E55760046410703FAB51AA52A953AE
:102E260012251864306009E557702E75570A8029F7
:102E3600900001122531FF64786004EFB458134303
:102E4600590175571074022553F553E43552F5525E
:102E56008007E5577003755708AB510553E553AA2C
:102E6600527002055214F9122518F55EC39461409A
:102E76000AE55ED3947A5003535EDF74D0255EF57F
:102E86005EC3940A400CE55E9411406D74F9255EAC
:102E9600F55EE55ED395575060435901855D6285C1
:102EA6005C61855B60855A5FAF577E00E4FCFDABD5
:102EB6005DAA5CA95BA85A1226EFC8ECC8C9EDC981
:102EC600CAEECACBEFCBE4FCFDFEEB255EF55DEE6C
:102ED6003AF55CED39F55BEC38F55AAF5DAE5CADB5
:102EE6005BFCAB62AA61A960A85FD31226A150035E
:102EF600022E5F435904022E5FE55920E003E48069
:102F06002DE55545564554601EAB51E55324FFF952
:102F1600E55234FFFAEBC0E0EAC0E0E9C0E0AB54AA
:102F2600AA55A95612274EE55930E20774FFFFFE4F
:102F3600FDFC22E559AF5DAE5CAD5BAC5A30E103FA
:042F460002269322AA
:1026EF00E88FF0A4CC8BF0A42CFCE98EF0A42CFC8A
:1026FF008AF0EDA42CFCEA8EF0A4CDA8F08BF0A408
:10270F002DCC3825F0FDE98FF0A42CCD35F0FCEB66
:10271F008EF0A4FEA9F0EB8FF0A4CFC5F02ECD392B
:0F272F00FEE43CFCEAA42DCE35F0FDE43CFC2298
:10273E00FAE6FB0808E6F925F0F618E6CA3AF6229C
:10274E00BB011A89828A83D0F0D0E0F8D0E0F9D0AC
:10275E00E0FAD0E0FBE8C0E0C0F00227CC5016E96A
:10276E00F8D083D082D0E0F9D0E0FAD0E0FBC0827E
:10277E00C0830227C3BBFE16E9F8D083D082D0E017
:0F278E00F9D0E0FAD0E0FBC082C0830227D52249
:10279D00D083D082F8E4937012740193700DA3A3CB
:1027AD0093F8740193F5828883E4737402936860DF
:0627BD00EFA3A3A380DFDF
:0927C300EBF608EAF608E9F6223B
:0927CC00EBF0A3EAF0A3E9F0220E
:0927D500EBF208EAF208E9F22235
:00000001FF
